:020000040000FA
:060000000000000058287A
:0800080000000000682B20201D
:1000100020202020202020202020282043202920AC
:1000200063206220702020203220302030203320B6
:1000300046207020722063203520722078202020F6
:10004000522065206C2065206120732065202020CF
:100050003120362046203820372033202020202011
:100060005820742061206C20320030002E003000B7
:1000700056206520722020203000330034002020DC
:100080004120632074202E204C206F2077202020D8
:100090005320742064202E2050206F2077202020B1
:1000A0004D206F2064206520542061206220312083
:1000B000203084005F30FF008001840AFF0B5C2841
:1000C000FF018B010630831603139F008312572212
:1000D0008613CB218312031390015A30E6006C2261
:1000E0000E22B227610EF039A7045222E02400004C
:1000F000861700000510643080220000861300007F
:100100000514B4222609CF002709D0002809D10000
:100110002909D200DC210030EB00FF30F6008B30E3
:10012000A200810182308316031381008312A03064
:100130008B00711EB3286D08B1006E08B20036271F
:10014000031CB2282414DD003D08C00060274F279F
:100150000318A3282230E421E02440085427023C5D
:10016000031D8D277112711DCA28241CC928ED2179
:100170003627031CC228DD003D08C00080274F271A
:100180000318BB28E024241040085427023C031D18
:100190008D277111C222481906290310D60CD50CDF
:1001A000D40CD30CD703D71FD628DC21570DAF00B2
:1001B000AF0E0330AF0526302F0784000008DF00A4
:1001C00053302F0784000008E0004F302F078400D1
:1001D0000008DE005E085F066005031906295E0858
:1001E0006005031DF8286008DE040130CD00FD28FD
:1001F0006009DE050030CD00FD285E08800057084C
:10020000CE006830CC000330CB0048150301230733
:1002100003196329A3030301650703191529E60BD5
:1002200015296508A704E501E024A41C2529861FDB
:100230001E29241A1E290830A4062A2924185929FF
:100240005722502503186E215929861F3029241A58
:100250005929A4140F30A4191E30BB21A301592918
:10026000241953295025031C5929C127031C592936
:10027000C6005427023C0319492946085427033C69
:100280000319492946085427043C03194929D22750
:1002900036293F08DD003D08C0006027E024241512
:1002A0000530E4005929502503185029E40B592939
:1002B0002411F1210301380703196329B80B6329BD
:1002C0001E27E0248D279928E0245025031864294F
:1002D0000800E0245025031C69290800B0007112B1
:1002E000BC01BE0100008617000005106421FA3031
:1002F0008022FA3080223C085427013EC600FA30A2
:1003000080220000861300000514963080226421AC
:100310000000861700000510C60B7F29711A9D2961
:10032000E0245025031C8E293C085427013E053C3F
:10033000031D053C5627BC007B29000086130000E6
:1003400005146D08BA006E08BB0030080F39BE04F2
:10035000A4193E16710E3039BC04D0260318B929F1
:10036000BB26031CB729AC27B227E02408000430C1
:10037000912A0330912AAF00000086170000051073
:1003800032308022000086130000051432308022B3
:10039000AF0BBC290800861F08003230BB21662243
:1003A000861FD5297C22BB21D3295025031CCF29A8
:1003B00002271430BB21CF298030D600D501D401CB
:1003C000D3011F30D7000800AA00C50A013045023A
:1003D000031D0800A4122416032AC50B0800A41646
:1003E0000800241E0800AB0B0800861F032A00002B
:1003F000861300000514A41A0B2A0F302A05AB003F
:100400000800A41A0B2A00008617000005102A0E07
:100410000F39AB0008002412A41208000430E200D7
:10042000E10107306207C127031C4F2A5427033C10
:10043000031D3A2A02308A0062038207342A2E2AD8
:10044000282A222A8316031385148312E1154F2AC2
:10045000831603138616831261154F2A831603131E
:1004600005158312E1144F2A83160313061683120F
:1004700061144F2A013E031D4D2A02308A00620397
:1004800082074B2A492A472A452AE515222A65155B
:10049000282AE5142E2A6514342AD227142AE20BBE
:1004A000112A08002708E5056509A705080000309E
:1004B00083160313850083124030831603138600CE
:1004C000831218308316031387008312A601A70135
:1004D000A801A901E02408008B138B1B6C2A0030B3
:1004E000522383120313AA3C0319080000305C2333
:1004F000AA302E2383120313ED26AC27E024080034
:10050000A000FA30A1006400852A862A872A882A5A
:10051000892A8A2A8B2A8C2AA10B832AA00B812A5A
:1005200008008B138B1B912AFC000130FE007C0815
:10053000FD000000861700000510643080220000D6
:10054000861300000514FA308022FD0B992AFA3038
:100550008022FA308022FA308022FA308022FA306B
:1005600080227E1C0800972A283094008C11831664
:10057000031380309400603091000A30930083129E
:100580000313080002308A0049088207C92AD52AC5
:10059000EA2A481DF02A8C118316031311148312C2
:1005A0000313CA010130C900F02A8C1DF02A8C11F6
:1005B000CB03CB1BE22A4A084C3E84000008930080
:1005C000CA0AF02A8316031311158312031302308B
:1005D000C900F02A8C1DF02A8C1148110030C90086
:0405E0000800202BC4
:10064000831203178C00831603178C130C15553077
:100650008D00AA308D008C140C1108008312031732
:100660008C00831603178C130C1555308D00AA309F
:100670008D008C140C11831603178C183D2B080069
:10068000831203178D00831603178C130C15553036
:100690008D00AA308D008C140C11831603178C1852
:1006A0004F2B0800831203178D00831603178C133A
:1006B0000C1483120C080800831203178D00080025
:1006C000831203178C000800831203178D0A080099
:1006D000FD00030E8301FC000A08FE008A010B11D5
:1006E000831203136400AC0B782BA30A9530AC0083
:1006F000EF0BD22C03308A006B0882078C2B942BD3
:10070000C62BD42BDA2B042C302C572C612C6B2CC1
:100710007A2C902C952CB92C061FC72C0B108B15FE
:100720000130EB00721171130B1C9C2B0B108B1101
:10073000513081000B117215061BAD2B7219A22BC3
:1007400000000000ED01F115F010F0150E30EC0086
:1007500070100430EB000330CB2CEF0AF01CD22CCD
:10076000701EBB2B7119BB2B711AC2247019C224C5
:10077000701571167012F40BD22CF30BD22CF010F2
:10078000701971157011FF30F600D22C7010061F11
:100790007014EB0ACA2CF01D542CF0110730EB003A
:1007A000D930A2000230CB2CEB0AF01DCA2C7117F5
:1007B0000130CB2C061FE02B701C4A2C0310E32BBE
:1007C0007018CB2B0314ED0DEE0DEC0BF52BFC305C
:1007D000F205F013701BF01770136E1A7017EE11FC
:1007E0006E1AEE150F30EE05FE2B0230EB00711B7A
:1007F000F0110430711B013E7113CB2C0530EB005E
:100800000530EC000430CB2C061F4A2CEC0B2E2CB0
:10081000FC30F10503307205F104F2156D08750224
:10082000031D162C6E0876020319F2110230F2191C
:10083000F900F90B252C701D212C71157016701103
:10084000252C701D71167015F1116D08F5006E08DC
:10085000F600F0140630EB002D30CB2C0430CB2CFE
:10086000033072050319382C023C031D3D2C422C29
:100870000230F300B930F400462C0130F300873029
:10088000F400462C0230F300D830F4000030EB00C6
:100890000130CB2CF1110030EB0070197115701183
:1008A000FF30F6004330CB2C8B30A2004A2C061FC1
:1008B000862CBA30A2000830EB000F30EC00ED01BE
:1008C000D02C061F682C03306C020319832C542C87
:1008D0000930EB00D02C061F752C0830EB000310FC
:1008E000ED0DEE0DEC0BD02C832C7214F2100A30AF
:1008F000EB00D02C061F542C0830EB000314ED0D38
:10090000EE0DEC0BD02C8B30A200FE2BD930A200C8
:100910000B30EB003130EC00ED01F7010430CB2C53
:10092000F8010C30EB008830A200F809780AA20721
:10093000F801061F9D2CF70ACD2C01307702031D0C
:10094000A32C0314A82C03307702031DAF2C031033
:10095000EC0BB22C7210F2148B30A200FE2B0000B4
:1009600000004A2CED0DEE0DF7010D30EB000130CB
:10097000CB2CEB30061F0F30F800A2070C30EB0039
:100980000130CB2C0000000008000630912A013015
:10099000EF00D22C0230EF00D22C0230EF00D22C2C
:1009A0000230EF002208810203180B150B1DD92C11
:1009B0006F2B7E088A007C0E8300FD0E7D0E0900E1
:1009C000261CE42C0715E52C0711A61CE92C87161C
:1009D000EA2C8712261DEE2C8714EF2C8710A61DFB
:1009E000F32C0717F42C0713261EF82C0714F92CE8
:1009F0000710A61EFD2C8717FE2C8713261F022D1D
:100A00000614032D0610A61F072D8614082D861028
:100A1000271C0C2D85160D2D8512A71C112D0615D2
:100A2000122D0611271D162D8615172D8611A71DAF
:100A30001B2D85151C2D8511A41C332D271E222D41
:100A40000616232D0612A71E272D0515282D051184
:100A5000271F2C2D86162D2D8612A71F312D8514AC
:100A6000322D85104F2D61183A2D271E392D06166F
:100A70003A2D0612E118412DA71E402D0515412DD6
:100A800005116119482D271F472D8616482D8612FE
:100A9000E1194F2DA71F4E2D85144F2D85100800ED
:100AA0000301261C562D071DE32D592D071D592D19
:100AB000E32D013EA61C5F2D871EE32D622D871EB0
:100AC000622DE32D013E261D682D871CE32D6B2D25
:100AD000871C6B2DE32D013EA61D712D071FE32DF5
:100AE000742D071F742DE32D013E261E7A2D071C41
:100AF000E32D7D2D071C7D2DE32D013EA61E832DAC
:100B0000871FE32D862D871F862DE32D013E261F8F
:100B10008C2D061CE32D8F2D061C8F2DE32D013E01
:100B2000A61F952D861CE32D982D861C982DE32D50
:100B3000013E271C9E2D851EE32DA12D851EA12D76
:100B4000E32D013EA71CA72D061DE32DAA2D061D92
:100B5000AA2DE32D013E271DB02D861DE32DB32DBB
:100B6000861DB32DE32D013EA71DB92D851DE32D57
:100B7000BC2D851DBC2DE32D013E271EC22D061E5A
:100B8000E32DC52D061EC52DE32D013EA71ECB2D41
:100B9000051DE32DCE2D051DCE2DE32D013E271F76
:100BA000D42D861EE32DD72D861ED72DE32D013E95
:100BB000A71FDD2D851CE32DE02D851CE02DE32DE9
:100BC000013E0310072EA418062EAF000C302F0292
:100BD000031DED2D611C052E032E0D302F02031D6C
:100BE000F42DE11C052E032E0E302F02031DFB2DCC
:100BF000611D052E032E0F302F02031D022EE11D55
:100C0000052E032E052E0430AF022F080314080012
:100C10002F260318080052263308A6043408A70418
:100C20003508A8043608A90408002F260318080070
:100C300052263309A6053409A7053509A805360942
:100C4000A90508002F260318080052263308A60617
:100C50003408A7063508A8063608A9060800DC00EF
:100C60000C305C02031D372E611C4F2E4D2E0D30B3
:100C70005C02031D3E2EE11C4F2E4D2E0E305C02F9
:100C8000031D452E611D4F2E4D2E0F305C02031D9E
:100C90004C2EE11D4F2E4D2E4F2E0314502E0310BF
:100CA0005C080800013EB301B401B501B6010314AC
:100CB000B30DB40DB50DB60DFF3E0310031D582E38
:100CC0000800B9000310B90DB90D080039088B13DD
:100CD0008B1B672E8A1500218A113A088A152D214F
:100CE00009218A113B088A152D2109218A113C0806
:100CF0008A152D2109218A113E088A152D218A1174
:100D00008B1708003908033E8B138B1B842E8A1522
:100D1000002114218A118B17BF00080039088B139A
:100D20008B1B8F2E8A15002114218A118B17AD0081
:100D3000080039088B138B1B9A2E8A150021142169
:100D40008A118B17AD008B138B1BA32E8A150921DB
:100D500014218A11AE008A15092114218A118B17DA
:100D6000BD008B138B1BB12E8A15092114218A110A
:100D70008B17BF0008002030A500AF012F086126A7
:100D8000992612270318CB2E8B138B1BC42E662695
:100D90008B1703140800AF0AA50BBE2E0310080022
:100DA0002030A500AF012F08612699262D083A02B0
:100DB000031DE82E2E083B02031DE82E3D083C02D1
:100DC000031DE82E3F083E02031DE82E0314080011
:100DD000AF0AA50BD32E031008002030A500AF01E9
:100DE000FC268B138B1BF12E2F0861266626AF0A7B
:100DF000A50BF42E8B170800FF30BA00BB00BC0116
:100E0000BE010800B0002030A500FC2625036126A5
:100E100099261F303F053006031D0F2F6626A50BB0
:100E2000062F08002D08FF3C031D1C2F2E08FF3C39
:100E3000031D1C2F03100800031408002030A50018
:100E4000AF012F08612699261227031C322F3D0877
:100E50005427023C031D322F3F0837020319322F5B
:100E60003F081526AF0AA50B212F08002030A5004A
:100E7000AF012F0861268E262D083106031D4F2F46
:100E80002F08612699262E083206031D4F2F3D0E8E
:100E900071060339031D4F2F3F0803140800AF0AE2
:100EA000A50B392F0310080007390800073908007F
:020EB000602FB1
:100EC00007308A004008542782076A2F6D2F702F41
:100ED000772F7A2F5D0808267F2F5D0822267F2F27
:100EE0005D0808265D08B7000430B8007F2F5D0854
:100EF00022267F2F5D0852263409E505772F08004A
:100F000007308A004008542782078A2F8C2F8C2FA5
:100F10008C2F8C2F5D08152608000430AF000030A0
:100F20002F07522383120313DB0025302F07840081
:100F300000085B020319A92F00302F075C238312DE
:100F4000031300088B138B1BA22F2E238312031372
:100F50008B17AF0B8F2F0800A601A701A801A901CD
:100F60008D2708000430AF0025302F0784000030A3
:100F70002F0752238312031380008403AF0BB72F74
:100F80000800C7002030A500AF012F086126822687
:100F90003F084702031DD22F2F08612699263D08DE
:0E0FA0000314D62FAF0AA50BC52F03100800AF
:10120000D8005B30D807D9010318D90A0930D907AB
:101210000800D80A031D0800D90A08000130D802C6
:1012200003180800D9030800831203135808031792
:101230008D000313590803178F0083168C170C14A5
:101240000000000083120C080313DA008316031752
:101250008C13831203135A080800DA008312031355
:10126000580803178D000313590803178F00031341
:101270005A0803178C0003018E0083168C170C1577
:10128000831203138B138316031755308D00AA3076
:101290008D008C14000000000C1183120313080051
:1012A00066206C20612073206820732074206120E8
:0612B000722074203A20B8
:02400E00763FFB
:00000001FF
